:1000000019C02BC02AC029C028C027C026C025C0BF
:1000100024C023C022C021C020C01FC01EC01DC0DC
:100020001CC01BC01AC019C018C017C016C015C00C
:1000300014C013C011241FBECFEFCDBFDFE3DEBF5E
:100040001FE3A0E0BFE3E8EAF7E002C005900D92ED
:10005000A430B107D9F702D1A0C3D2CF2F923F92DB
:100060004F925F926F927F928F929F92AF92BF92C8
:10007000CF92DF92EF92FF920F931F93CF93DF9374
:10008000CDB7DEB7AA97CDBFDEBF062F172F8AA741
:1000900099A72BEA3AEA4AE25FE3C62ED72EE82E6A
:1000A000F92EC701B60116D3C62ED72EE82EF92E8B
:1000B00020E030E040E85FE3862E972EA82EB92E90
:1000C000C501B401B9D181150CF4AFC020E030E016
:1000D00040E05FE3402E512E6AA479A4C301B2012F
:1000E000F9D2862E972EA82EB92E20E03FEF4FE7AB
:1000F00057E469837A838B839C8369817A818B81BE
:100100009C81E4D2811509F0DCF420E030E04FE777
:1001100053E4CD82DE82EF82F8866D817E818F810D
:100120009885D4D2811511F00CF072C0C986DA8698
:10013000EB86FC8669857A858B859C85E9D176C0BE
:1001400020E030E04AE754E40D871E876F86788A06
:100150006D857E858F85988973D1C62ED72EE82E22
:10016000F92E20E030E04AEF53E4698B7A8B8B8BD9
:100170009C8B69897A898B899C89ACD2062F172F31
:100180008D83998320E03FEF4FE757E46D8B7E8BA3
:100190008F8B988F6D897E898F89988D97D28115E5
:1001A00009F07CF4098F1A8F8D818B8F89818C8F58
:1001B000698D7A8D8B8D9C8DABD1CB010197F1F739
:1001C00037C020E030E040E251E4C9A2DAA2EBA25D
:1001D000FCA269A17AA18BA19CA17CD26DA37EA374
:1001E0008FA398A76DA17EA18FA198A591D1262E4E
:1001F000372E21143104E1F022E330E0C9010197E8
:10020000F1F781E0281A310821143104B9F710C040
:100210008D8E9E8EAF8EB8A26D8D7E8D8F8D98A1A6
:1002200077D1CB010197F1F703C061E06A95F1F74F
:10023000AA96CDBFDEBFDF91CF911F910F91FF90A6
:10024000EF90DF90CF90BF90AF909F908F907F9076
:100250006F905F904F903F902F9008950F2EF8EA87
:10026000EF2EF7E8FF2EF02D0DE110E1CEE9D7E8F3
:10027000DFD0C8010197F1F770D07CD089919991B6
:1002800086D0CE15DF05A1F7F1CF61E088E096E0DA
:1002900061D0E0E0F6E0838580FFFDCFE0E0F6E0AE
:1002A00081E08387808991890895CF93C82F883012
:1002B00010F0CF910895682F82E094E02AD06C2F3F
:1002C00086E094E026D08C2F90E064E0805F9B4F26
:1002D00020D062E080E096E029D064E082E096E001
:1002E00018D0E7CF883008F00895682F86E096E0B0
:1002F0002BD060E080E096E00CD0089586E096E098
:1003000005D060E080E096E011D00895FC011082F5
:100310000895E82FF92F81E090E002C0880F991F1F
:100320006A95E2F76081682B60830895E82FF92FC2
:1003300081E090E002C0880F991F6A95E2F78095EE
:100340009081892380830895E82FF92F8081862B5F
:1003500080830895FC016083089561E080E094E06B
:10036000D8DF63E080E294E0D4DF62E080E294E0F2
:10037000D0DF089561E084E094E0CBDF63E084E2C5
:1003800094E0C7DF62E084E294E0C3DF0895CF9297
:10039000DF92EF92FF92BC0180E090E0E5D0E09127
:1003A000003FF091013FC62ED72EE82EF92EC7014F
:1003B000B601099561E084E094E0B8DF63E084E28F
:1003C00094E0B4DF62E084E294E0B0DFFF90EF906D
:1003D000DF90CF90089587E068DF87E083DF08959E
:1003E0000F931F93CF93DF93F6DFE091023FF091DD
:1003F000033F87E00995082F192F80DFECDFE0919C
:10040000023FF091033F87E00995C82FD92F76DF8F
:1004100091E0C017D10708F490E081E0C115D24007
:1004200008F480E08923DF91CF911F910F91089507
:10043000D7DF8115E9F30895D4D008F481E0089559
:100440000CD00AC102D140F0F9D030F021F45F3F66
:1004500019F0EBC0511134C1EEC00FD198F39923BC
:10046000C9F35523B1F3951B550BBB27AA27621778
:100470007307840738F09F5F5F4F220F331F441FBD
:10048000AA1FA9F333D00E2E3AF0E0E830D09150F5
:100490005040E695001CCAF729D0FE2F27D0660FE2
:1004A000771F881FBB1F261737074807AB07B0E821
:1004B00009F0BB0B802DBF01FF2793585F4F2AF037
:1004C0009E3F510568F0B1C0FBC05F3FECF3983E22
:1004D000DCF3869577956795B795F7959F5FC9F794
:1004E000880F911D9695879597F90895E1E0660F1D
:1004F000771F881FBB1F621773078407BA0720F096
:10050000621B730B840BBA0BEE1F88F7E0950895FE
:10051000BCD088F09F5790F0B92F9927B751A0F021
:10052000D1F0660F771F881F991F1AF0BA95C9F787
:1005300012C0B13081F0C3D0B1E00895C0C0672FC0
:10054000782F8827B85F39F0B93FCCF38695779537
:100550006795B395D9F73EF4909580957095619520
:100560007F4F8F4F9F4F0895E89409C097FB3EF44B
:1005700090958095709561957F4F8F4F9F4F9923F0
:10058000A9F0F92F96E9BB279395F695879577956E
:100590006795B795F111F8CFFAF4BB0F11F460FF2E
:1005A0001BC06F5F7F4F8F4F9F4F16C0882311F086
:1005B00096E911C0772321F09EE8872F762F05C09A
:1005C000662371F096E8862F70E060E02AF09A9535
:1005D000660F771F881FDAF7880F9695879597F92A
:1005E0000895990F0008550FAA0BE0E8FEEF1616C4
:1005F0001706E807F907C0F012161306E407F50717
:1006000098F0621B730B840B950B39F40A2661F08A
:10061000232B242B252B21F408950A2609F4A1402D
:10062000A6958FEF811D811D089597F99F6780E83A
:1006300070E060E008959FEF80EC089500240A9434
:100640001616170618060906089500240A941216AD
:100650001306140605060895092E0394000C11F4E0
:10066000882352F0BB0F40F4BF2B11F460FF04C08D
:100670006F5F7F4F8F4F9F4F089557FD9058440FE6
:10068000551F59F05F3F71F04795880F97FB991FF1
:1006900061F09F3F79F087950895121613061406AE
:1006A000551FF2CF4695F1DF08C01616170618063B
:1006B000991FF1CF86957105610508940895E89416
:1006C000BB2766277727CB0197F908958ADF08F4BF
:1006D0008FEF08950BD0C0CFB1DF28F0B6DF18F050
:1006E000952309F0A2CFA7CF1124EACFC6DFA0F34C
:1006F000959FD1F3950F50E0551F629FF001729FB7
:10070000BB27F00DB11D639FAA27F00DB11DAA1FD5
:10071000649F6627B00DA11D661F829F2227B00D22
:10072000A11D621F739FB00DA11D621F839FA00DAD
:10073000611D221F749F3327A00D611D231F849FFD
:10074000600D211D822F762F6A2F11249F57504054
:100750008AF0E1F088234AF0EE0FFF1FBB1F661FEF
:10076000771F881F91505040A9F79E3F510570F0A8
:100770005CCFA6CF5F3FECF3983EDCF38695779590
:100780006795B795F795E7959F5FC1F7FE2B880FA3
:0E079000911D9695879597F90895F894FFCFDF
:0A079E00FA00F401EE02E803E204A1
:0407A8002E004501D9
:00000001FF
